:100000000C9476070C94BA070C94BA070C94BA07B0
:100010000C94BA070C94BA070C94BA070C94BA075C
:100020000C94BA070C94BA070C94FE120C94D013DB
:100030000C94BA070C94BA070C94BA070C94BA073C
:100040000C94BA070C94AA2C0C94BA070C94BA0717
:100050000C94BA070C94A2220C94BA070C94BA0719
:100060000C94BA070C94BA070C94BA070C94BA070C
:100070000C94BA070C94BA070C94BA070C94BA07FC
:100080000C94BA070C94BA070C94BA070C94BA07EC
:100090000C94BA070C94BA070C94BA070C94BA07DC
:1000A0000C94BA070C94BA070C94BA073D145F1469
:1000B0004D155F144D15A414C7144D151C152F159F
:1000C00076187618A518A518E81826193F1B3F1BA7
:1000D0003F193F1B401A401A131B3F1B3F1B2A1B93
:1000E0000147024701470247012102210128022856
:1000F0000001470247014702470120022001280270
:1001000028000147024701470247011F021F01283B
:100110000228000147024701470247011E021E0153
:1001200028022800000001C002C003C004C005C0AE
:10013000018C028C2E004C002900E1003582000069
:100140001E00140004001D0034004D821F001A0020
:1001500015001B00E1042A712000090016000600AA
:1001600050002C7221001300170019004F004A00A4
:1001700022000A00070005000000E20050000254BF
:100180000000007F000001204F00025400000077B3
:100190000000E20023000D000B000E000000E6004E
:1001A00024000F001100100052004B002500180021
:1001B000080036005100287226001C000C00370091
:1001C0002F002B71270033001200387130004E834E
:1001D0002D0031003400E500008200002E004C00AC
:1001E0002900E100358200001E00140004001D00FB
:1001F00034004D821F001A0016001B00E1042A7112
:10020000200008000700060050002C722100150095
:10021000090019004F004A00220017000A000500DB
:100220000000E200500002540000007F00000120A6
:100230004F000254000000770000E20023001C0081
:100240000B0011000000E600240018000D00100053
:1002500052004B0025000C000E00360051002872A1
:10026000260012000F0037002F002B71270013000B
:100270003300387130004E832D0031003400E5002A
:1002800000820000010001000100010001000000E7
:100290003A001E0220022202010001003B001F0260
:1002A00021022302010001003C002F0226022F0040
:1002B000010001003D003002270230000100010072
:1002C0003E0031023500350200000100010001004E
:1002D0000000010000000100010001000000010019
:1002E000000001003F005200510024020000010004
:1002F0004000240021001E000100010041002500F3
:1003000022001F00370001004200260023002000C9
:1003100027000100430025022E0231002E000100BB
:100320004400450001000100010000000000000041
:100330000000000000000000000006200220000075
:100340000000010000000720032000000000010061
:100350000000000004200000000001000000000078
:100360000520000000000100000000000000000067
:10037000000001000000000000000000000001007B
:10038000000000000000000000000100000000006C
:10039000000000000000010000000000000000005C
:1003A000000001000000000000000000000001004B
:1003B000000000000000000000000100000000003C
:1003C000000000000000010000000000000000002C
:1003D000000000000A002530313662003A20002576
:1003E000303258000A722F632030313233343536C0
:1003F0003738394142434445460A000A0025303225
:100400005800626F756E6365213A20006C656674F2
:1004100020736964652061747461636865640A00AF
:100420006C6566742073696465206E6F74207265F4
:1004300073706F6E64696E670A00747279696E67B3
:1004400020746F207265736574206D637032333071
:1004500031380A005B735D004B6579626F617264CD
:100460002073746172742E0A005B575D005B535DEC
:10047000005B525D005B445D005B435D001603451D
:1004800000720067006F0044006F00780020004594
:10049000005A00000016034500720067006F004418
:1004A000006F007800200045005A00000004030996
:1004B0000409028D00050100A0FA090400000103EF
:1004C000010100092111010001223F0007058103FC
:1004D00008000A09040100010301020009211101B9
:1004E0000001224D000705820308000A09040200EA
:1004F0000103000000092111010001223600070557
:10050000830308000A090403000203000000092114
:1005100011010001222000070584032000010705C6
:100520000403200001090404000103000000092164
:100530001101000122390007058503100001120195
:10054000100100000008EDFE071301000102000188
:1005500005010906A101050719E029E71500250194
:100560009508750181020508190129059505750190
:10057000910295017503910105071900297715006E
:100580002501957875018102C00631FF0974A1012A
:100590000975150025FF952075088102097615005B
:1005A00025FF952075089102C005010980A10185EC
:1005B0000216010026B7001A01002AB7007510952F
:1005C000018100C0050C0901A10185031601002667
:1005D0009C021A01002A9C02751095018100C00539
:1005E000010902A1010901A1000509190129051547
:1005F00000250195057501810295017503810105AD
:1006000001093009311581257F9502750881060998
:10061000381581257F950175088106050C0A380279
:100620001581257F950175088106C0C00501090661
:10063000A101050719E029E71500250195087501B5
:1006400081029501750881010508190129059505A3
:10065000750191029501750391010507190029FFA4
:10066000150025FF950675088100C00A0025303267
:100670005820006B6579626F6172645F7265706F9C
:1006800072743A20000A0025303258006B65796296
:100690006F6172645F7365745F6C65643A200064B7
:1006A000656C5F6B65795F6269743A2063616E2780
:1006B000742064656C3A20253032580A0061646405
:1006C0005F6B65795F6269743A2063616E2774209D
:1006D0006164643A20253032580A00646F6E652EDA
:1006E0000A00626F6F676D61676963207363616E93
:1006F0003A202E2E2E2000290A002575002F0025D5
:1007000075005D2800256400200025640020002578
:10071000640020002564007C0025303258006D6F95
:100720007573656B6579205B62746E7C78207920C7
:100730007620685D287265702F61636C293A205BB2
:10074000006D6B5F776865656C5F74696D655F747C
:100750006F5F6D6178203D2025640A006D6B5F77C7
:100760006865656C5F6D61785F7370656564203D79
:100770002025640A006D6B5F74696D655F746F5F3F
:100780006D6178203D2025640A006D6B5F6D617896
:100790005F7370656564203D2025640A006D6B5FA2
:1007A000696E74657276616C203D2025640A006D67
:1007B0006B5F64656C6179203D2025640A006D6B78
:1007C0005F776865656C5F74696D655F746F5F6D99
:1007D0006178203D2025640A006D6B5F7768656550
:1007E0006C5F6D61785F7370656564203D20256482
:1007F0000A006D6B5F74696D655F746F5F6D617822
:10080000203D2025640A006D6B5F6D61785F737019
:10081000656564203D2025640A006D6B5F696E7418
:10082000657276616C203D2025640A006D6B5F6403
:10083000656C6179203D2025640A000A0025750059
:10084000363A20776865656C5F74696D655F746FB3
:100850005F6D61783A20000A00257500353A2077EF
:100860006865656C5F6D61785F73706565643A207B
:10087000000A00257500343A2074696D655F746F55
:100880005F6D61783A20000A00257500333A206DCB
:1008900061785F73706565643A20000A0025750011
:1008A000323A20696E74657276616C286D73293AEC
:1008B00020000A00257500313A2064656C617928B2
:1008C0002A31306D73293A20000A092D2056616CB7
:1008D000756573202D0A004D3E004D25643E2000B5
:1008E0003F007365742064656661756C740A00432B
:1008F0003E200077686572652064656C74613A20FB
:10090000637572736F723D25642C20776865656C22
:100910003D25640A53656520687474703A2F2F650D
:100920006E2E77696B6970656469612E6F72672FCF
:1009300077696B692F4D6F7573655F6B6579730AA6
:10094000000A092D204D6F7573656B6579202D0A9E
:100950004553432F713A09717569740A313A096434
:10096000656C6179282A31306D73290A323A096938
:100970006E74657276616C286D73290A333A096D5D
:1009800061785F73706565640A343A0974696D65EE
:100990005F746F5F6D61780A353A09776865656CD9
:1009A0005F6D61785F73706565640A363A097768D0
:1009B00065656C5F74696D655F746F5F6D61780A02
:1009C0000A703A097072696E742076616C7565738D
:1009D0000A643A097365742064656661756C7473A2
:1009E0000A75703A092B310A646F776E3A092D3116
:1009F0000A706775703A092B31300A7067646F7737
:100A00006E3A092D31300A0A7370656564203D2005
:100A100064656C7461202A206D61785F7370656510
:100A200064202A2028726570656174202F20746903
:100A30006D655F746F5F6D6178290A003F004D3E00
:100A40002000433E20004C25640A000A092D204363
:100A50006F6E736F6C65202D0A4553432F713A09F1
:100A6000717569740A6D3A096D6F7573656B657997
:100A70000A000A092D204D61676963202D0A643A36
:100A80000964656275670A783A096465627567206A
:100A90006D61747269780A6B3A09646562756720E2
:100AA0006B6579626F6172640A6D3A09646562759B
:100AB00067206D6F7573650A763A0976657273699A
:100AC0006F6E0A733A097374617475730A633A0935
:100AD000636F6E736F6C65206D6F64650A302D34C3
:100AE0003A096C61796572302D34284631302D46D3
:100AF00034290A506175733A09626F6F746C6F61C3
:100B00006465720A653A09656570726F6D0A6E3ABE
:100B1000094E4B524F0A7A3A09736C656570204C46
:100B2000454420746573740A000A002575002E6E12
:100B30006B726F3A20000A002575002E7377617082
:100B40005F6261636B736C6173685F6261636B7337
:100B5000706163653A20000A002575002E73776185
:100B6000705F67726176655F6573633A20000A00A3
:100B70002575002E6E6F5F6775693A20000A0025A3
:100B800075002E737761705F72616C745F72677548
:100B9000693A20000A002575002E737761705F6C3A
:100BA000616C745F6C6775693A20000A00257500F6
:100BB0002E636170736C6F636B5F746F5F636F6ED6
:100BC00074726F6C3A20000A002575002E737761ED
:100BD000705F636F6E74726F6C5F636170736C6F64
:100BE000636B3A20000A0025303258006B65796D3E
:100BF00061705F636F6E6669672E7261773A20007D
:100C00000A002575002E6D6F7573653A20000A0085
:100C10002575002E6B6579626F6172643A20000A57
:100C2000002575002E6D61747269783A20000A0003
:100C30002575002E656E61626C653A20000A0025FC
:100C40003032580064656275675F636F6E6669670E
:100C50002E7261773A20000A00257500646566618E
:100C6000756C745F6C617965723A20003F004E4B81
:100C7000524F3A206F66660A004E4B524F3A206F31
:100C80006E0A0074696D65725F636F756E743A20E9
:100C90002530346C580A006B6579626F6172645F4D
:100CA0006E6B726F3A2025580A006B6579626F612E
:100CB00072645F69646C653A2025580A006B657937
:100CC000626F6172645F70726F746F636F6C3A20F1
:100CD00025580A00686F73745F6B6579626F617283
:100CE000645F6C65647328293A2025580A000A0954
:100CF0002D20537461747573202D0A004743433AC5
:100D000020342E392E33204156522D4C4942433A3D
:100D100020312E382E31204156525F415243483AFD
:100D200020617672350A004F5054494F4E533A2095
:100D30004C55464120424F4F544D41474943204D69
:100D40004F5553454B45592045585452414B4559F1
:100D500020434F4E534F4C4520434F4D4D414E4441
:100D6000204E4B524F203531320A004255494C44F7
:100D70003A20333064623330302D646972747920E4
:100D80002830373A35373A3335204A616E203237CA
:100D90002032303136290A005649443A203078460C
:100DA000454544284572676F446F7820455A29208D
:100DB0005049443A20307831333037284572676FD4
:100DC000446F7820455A29205645523A20307830D1
:100DD0003030310A00444553433A20742E6D2E6B57
:100DE0002E206B6579626F617264206669726D771F
:100DF00061726520666F72204572676F646F780A52
:100E0000000A092D2056657273696F6E202D0A0045
:100E10000A6D6F7573653A206F66660A000A6D6F1A
:100E20007573653A206F6E0A000A6B6579626F61AF
:100E300072643A206F66660A000A6B6579626F61B8
:100E400072643A206F6E0A000A6D61747269783AB2
:100E5000206F66660A000A6D61747269783A206FC5
:100E60006E0A000A64656275673A206F6E0A000AAE
:100E700064656275673A206F66660A000A0A626FE7
:100E80006F746C6F616465722E2E2E2000433E20BD
:100E9000006565636F6E6669673A0A00536C656545
:100EA00070204C454420746573740A0000000000F3
:100EB00000000000000000010204060A0F17202CA9
:100EC0003A4A5D71879DB3C7DAE9F5FCFFFCF5E9A5
:100ED000DAC7B39D87715D4A3A2C20170F0A0604C2
:100EE00002010000000000000000000011241FBEED
:100EF000CFEFDAE0DEBFCDBF04B603FE24C08091A1
:100F0000F9019091FA01A091FB01B091FC018730A9
:100F1000904BA740B04BB9F41092F9011092FA012E
:100F20001092FB011092FC0114BE84B7877F84BF2E
:100F300088E10FB6F89480936000109260000FBEB5
:100F4000E0E0FFE3099511E0A0E0B1E0E0EFFCE5AF
:100F500002C005900D92AA33B107D9F711E0AAE3B8
:100F6000B1E001C01D92A93FB107E1F70E94361020
:100F70000C94762E0C940000FF93EF93E0913A01CD
:100F8000F0913B01309709F00995EF91FF91089599
:100F9000FC018591803011F0EFDFFBCF0895FF2732
:100FA000E0E230E247FF0CC0419597FF09C0EDE257
:100FB0006095709580959095611D711D811D911DA5
:100FC00027FF02C0219530E350E2AA27660F771F62
:100FD000881F991FAA1FA41710F0A41B63955A9588
:100FE000A9F7AA3008F0A95FA05DAF93F39561154A
:100FF00071058105910541F7ED3211F4EF93F395F9
:10100000F21718F43F93F395FBCF8F91B5DFFA9564
:10101000E1F70895E991F9918591803021F08532C9
:1010200019F0AADFF9CF089520E0E89455915532E0
:10103000C1F3503311F4689455915A3348F4505326
:1010400090F3220F022E220F220F200D250FF4CF36
:101050000EF4219589919991533619F3533729F15B
:10106000533559F1BC0188279927E8945C3621F45F
:101070008991999168945591543639F446EF7EF0F0
:1010800077FF0DC08FEF9FEF0AC055374AE039F068
:10109000583540E121F0523642E009F00895FF93BF
:1010A000EF937DDFEF91FF91B7CFFF93EF93FC01BB
:1010B00081918030B9F360DFFBCFFF93EF9368DF5E
:1010C000F1CFDF93CF93CDB7DEB72596A3DFCF91D6
:1010D000DF910895FC01623021F128F4662349F084
:1010E000613071F036C0643041F108F1653059F17A
:1010F00030C08281882311F085EE0CC085EE0EC0D1
:101100008281882351F085EE0E94131785EE0E949C
:10111000DB1783EE0E9413171CC083EE0E94DB17BF
:1011200018C08281811115C083E191E00895828108
:1011300081110FC082E091E008958281811109C080
:1011400081EF90E008958281811103C080EE90E0EC
:10115000089580E090E0089580E090E00895609127
:10116000BC017091BD018091BE019091BF010E94B0
:10117000A12156985E9825982D9826982E98279804
:101180002F98823019F0833021F00895259A2D9AF6
:101190000895269A2E9A08958FEA98E0892B11F0E7
:1011A0000E94AF0880E090E0089556985E982598D8
:1011B0002D9826982E9827982F988FEF90E090934F
:1011C00089008093880090938B0080938A0090938D
:1011D0008D0080938C00259A2D9A2FEF80E792E066
:1011E000215080409040E1F700C00000269A2E9ADE
:1011F0002FEF80E792E0215080409040E1F700C05F
:101200000000279A2F9A2FEF80E792E0215080402C
:101210009040E1F700C0000025982D982FEF80E75F
:1012200092E0215080409040E1F700C000002698F5
:101230002E982FEF80E792E0215080409040E1F718
:1012400000C0000027982F9856985E9825982D98F2
:1012500026982E9827982F98089589EA80938000E1
:1012600089E08093810024982C983F988AB18F74EC
:101270008AB96E98479A8BB1806B8BB9769A0E9427
:10128000D5088CEA98E0892B11F00E94AC0880E028
:1012900090E0089580E28093000180913C018111EB
:1012A0000EC00E94990981E080933C012FEF83EDED
:1012B00090E3215080409040E1F700C0000080E4BE
:1012C0000E949F098093000181112EC00E94C909CC
:1012D00080930001811128C00E94C90980930001F8
:1012E000811122C08FE30E94C909809300018111FE
:1012F0001BC00E94C10980E40E949F0980930001E5
:10130000811112C08CE00E94C909809300018111F3
:101310000BC00E94C90980930001811105C08FE3B1
:101320000E94C909809300010E94C10980910001B7
:1013300008951092B9008AE08093B800089594EA65
:101340009093BC009091BC0097FFFCCF9091B900A6
:10135000987F983021F0903111F081E008958093CA
:10136000BB0084E88093BC008091BC0087FFFCCF69
:101370008091B900887F883111F0803471F780E066
:10138000089584E98093BC008091BC0084FDFCCF6B
:1013900008958093BB0084E88093BC008091BC00DA
:1013A00087FFFCCF9091B900987F81E0983209F4D3
:1013B00080E0089584E88093BC008091BC0087FFA2
:1013C000FCCF8091BB00089580910001811115C070
:1013D00080E40E949F098093000181110CC082E18A
:1013E0000E94C90980930001811105C08FEF0E94FE
:1013F000C909809300010E94C10984B1807F84B92A
:1014000085B1807F85B98AB1837F8AB98BB1837FAB
:101410008BB93E98469808950E944A09809300012E
:101420000E94E40980B38C7080BB81B3836F81BB61
:10143000AEE3B1E0ECE4F1E08EE08E0F11921D928C
:101440008E13FCCF8DE299E0892B11F00C942D09BD
:1014500008959F92AF92BF92CF92DF92EF92FF9248
:101460000F931F93CF93DF93809100018823E1F0C6
:1014700080913D018F5F80933D01811115C08AE30A
:1014800094E00E94C8070E944A09809300018823C3
:1014900029F080E294E00E94C80706C08CE094E046
:1014A0000E94C8070E94D5080EE311E0C0E0D0E01A
:1014B000BB24B39482E0A82ECC24C394D12C2DEF6E
:1014C000E22E23E0F22EC730D10500F58091000115
:1014D000811164C080E40E949F0980930001811102
:1014E00012C082E10E94C9098093000181110BC0E2
:1014F000C6010C2E01C0880F0A94EAF780950E945D
:10150000C909809300010E94C10948C0CA30A1F0F6
:1015100028F4C83059F0C93061F005C0CC3089F0EA
:1015200070F0CD3089F0209A289810C0219A29981F
:101530000DC0229A2A980AC0239A2B9807C0529A63
:1015400001C0539A5B9802C03E9A469890EA9A95D9
:10155000F1F79FB1799902C082E001C080E09170FB
:101560009B25982B7C9902C084E001C080E0892BE8
:101570007D9902C038E001C030E0832B7E9902C023
:1015800020E101C020E0822B9FB19095991F9927FF
:10159000991F9295990F907E892B10C08091000120
:1015A000811174C080E40E949F0980930001882308
:1015B00009F459C0912C0E94C109892DF80190812C
:1015C000981739F1808380910101882301F180917E
:1015D000D70180FF04C082E094E00E94C807809198
:1015E000D70180FF0CC0809101011F928F93FF9261
:1015F000EF920E9461080F900F900F900F908091D2
:10160000D70180FF04C08BEF93E00E94C807A0922F
:1016100001010E94E40921960F5F1F4FCE30D105D2
:1016200009F051CF809101018823B1F0815080935E
:101630000101882339F08FE99FE00197F1F700C09D
:1016400000000AC0ACE4B1E0EEE3F1E0CF01825F5C
:1016500091919D938E13FCCF8CEC98E0892BC1F077
:101660000E94CC0815C083E10E94C9098093000143
:101670008111A0CF81E40E949F0980930001811114
:1016800099CF0E94DA09982E909495CF80E096CF5A
:1016900081E0DF91CF911F910F91FF90EF90DF904C
:1016A000CF90BF90AF909F900895E82FF0E0E45B5B
:1016B000FE4F80810895CF92DF92EF92FF920F93B9
:1016C0001F93CF93DF9384EE93E00E94C8078CE4CE
:1016D000E82E81E0F82EC0E0D0E09FEDC92E93E027
:1016E000D92E06ED13E0DF93CF93DF92CF920E94C5
:1016F00061088CED93E00E94C807F70181917F019A
:1017000090E00E9407229F938F931F930F930E9454
:10171000610884ED93E00E94C80721968DB79EB7BB
:1017200008960FB6F8949EBF0FBE8DBFCE30D10580
:10173000D1F6DF91CF911F910F91FF90EF90DF9045
:10174000CF9008958B3B910578F4883A910540F548
:10175000853A9105D0F48430910508F0B1C081300C
:10176000910509F4ADC06BC0803E910508F467C0D7
:10177000883E910508F4A4C09C01205F3109203106
:10178000310508F05CC090650895853A910509F42B
:1017900059C0863A910509F058C082E890E408954E
:1017A000883A910509F454C0893A910509F453C067
:1017B0008A3A910509F452C08B3A910509F451C057
:1017C0008C3A910509F450C08D3A910509F44FC047
:1017D000803B910509F44EC08E3A910509F44DC045
:1017E0008F3A910509F44CC0813B910509F44BC037
:1017F000823B910509F44AC0833B910509F449C035
:10180000843B910509F448C0853B910509F447C024
:10181000863B910509F446C0873B910509F445C014
:10182000883B910509F444C0893B910509F443C004
:101830008A3B910509F442C080E094E4089580E079
:1018400090E0089581E890E4089583E890E4089595
:1018500082EE94E4089589EE94E408958AEE94E487
:10186000089585EB94E4089586EB94E4089587EB5E
:1018700094E408958CEC94E408958DEC94E4089538
:1018800083E895E408958AE895E4089582E995E46B
:10189000089584E995E4089581E296E4089583E249
:1018A00096E4089584E296E4089585E296E4089526
:1018B00086E296E4089587E296E408958AE296E443
:1018C0000895089596E0799FF001112494E5899F89
:1018D000E00DF11D1124E60FF11DEE0FFF1FEC5C72
:1018E000FE4F859194910895880F991FFC01EC5546
:1018F000F040859194910895880F991FFC01EC5D4B
:10190000FE4F85919491089526E0729FF001112475
:1019100044E5849FE00DF11D1124E60FF11DEE0F4B
:10192000FF1FEC5CFE4F859194919C013A95211527
:101930004FE1340708F41AC13F512115304120F41A
:101940009F700E947C0C08959C01305321153041FA
:1019500018F49927906C0895811520E5920769F491
:101960000E94611B4FEF84E39CE041508040904017
:10197000E1F700C000000C94C722813020E59207F7
:1019800031F48091D70181608093D70108959C0143
:1019900030552115304108F051C0292F33272F70C1
:1019A000332721303105D9F4AC014370552702C0EB
:1019B000220F331F4A95E2F73C68AC0164E0440F04
:1019C000551F6A95E1F744275370242B352B73E09C
:1019D000880F991F7A95E1F7807699271DC02230EC
:1019E000310529F4982F8827816F906A0895233054
:1019F0003105A9F4AC014370552721E030E002C065
:101A0000220F331F4A95E2F73C6843E0880F991F85
:101A10004A95E1F7807E9770822B932B08952430AE
:101A20003105E1F4AC014370552721E030E002C0FC
:101A3000220F331F4A95E2F73A68E7CF9C013057EF
:101A40002115304118F49F70906208959C01305820
:101A50002115304118F49F70906A0895803E9105D9
:101A6000E0F4803C910558F58133910509F46FC08D
:101A700048F48932910509F463C08A32910509F46A
:101A80006DC072C089339105E9F082389105D1F0BB
:101A90008533910509F44DC067C0833E910581F1FE
:101AA00038F4803E9105B9F0823E9105D9F05CC0D2
:101AB000863E910561F1873E9105A1F155C00E94D6
:101AC000740C08952091EA0120FD02C021FF4CC052
:101AD00080EE90E049C08091EA0180FFF9CF89E370
:101AE00090E042C08091EA0182FF0EC08091EA013D
:101AF00084FF03C080E090E037C083EE90E034C004
:101B00008091EA0182FFF2CF82EE90E02DC08091B9
:101B1000EA0183FF0BC08091EA0184FDEBCF87EEE1
:101B200090E022C08091EA0183FFF5CF86EE90E03D
:101B30001BC08091EA0185FF07C089E290E014C0D4
:101B40008091EA0185FFF9CF85E390E00DC0809197
:101B5000EA0186FF07C08AE290E006C08091EA01B0
:101B600086FFF9CF81E390E00E94A20B08950895CB
:101B700080916D0108959FB7F89410925C019FBF0A
:101B80009091F001943009F057C09091E9009F7056
:101B90003091EC00232F217030FD20E8922B24E0BF
:101BA0002093E9002091EB0020FF43C02091EE003C
:101BB00027FF3FC020915A01222321F02091E80005
:101BC00025FF37C010925A0126E03091E80035FD1C
:101BD00015C03091F001343061F53091EB0035FDE6
:101BE00028C0215021F481E080935A0122C0EFE9FE
:101BF000FFE03197F1F700C00000E7CF8093F100DC
:101C00008091E80085FD0AC08091E80080FFFCCF4C
:101C10008091E8008E778093E80006C08FB7F89433
:101C200021E020935C018FBF9F709093E90080E0DA
:101C300008959F709093E9008FEF0895CF93DF93FD
:101C400000D01F92CDB7DEB79C018091F0018430A7
:101C500019F593E099833B832A839093E9008FEFF2
:101C60009091E800815095FD06C095ED9A95F1F7A9
:101C700000008111F5CF8091E80085FF0DC040E0A4
:101C800050E063E070E0CE0101960E94EE1080917A
:101C9000E8008E778093E8000F900F900F90DF910F
:101CA000CF910895CF93DF9300D01F92CDB7DEB7C9
:101CB0002091F001243021F522E029839B838A833F
:101CC00083E08093E9008FEF9091E800815095FDCB
:101CD00006C095ED9A95F1F700008111F5CF80913E
:101CE000E80085FF0DC040E050E063E070E0CE0109
:101CF00001960E94EE108091E8008E778093E800B4
:101D00000F900F900F90DF91CF9108952091F001E7
:101D10002430F1F422E02093E9002FEF3091E80025
:101D2000215035FD06C035ED3A95F1F7000021113F
:101D3000F5CF2091E80025FF0BC040E050E065E0C2
:101D400070E00E94EE108091E8008E778093E800AA
:101D50000895CF93DF932091F001243009F048C01B
:101D6000EC0180910C018823E1F080910D01882322
:101D7000C1F085E08093E9008FEF9091E8008150F9
:101D800095FD06C095E19A95F1F700008111F5CF18
:101D90008091E80085FF2CC040E050E060E170E0F9
:101DA00017C081E08093E9008FEF9091E8008150A7
:101DB00095FD06C095ED9A95F1F700008111F5CFDC
:101DC0008091E80085FF14C040E050E068E070E0DA
:101DD000CE010E94EE108091E8008E778093E8009B
:101DE00080E1FE01ADE5B1E001900D928A95E1F749
:101DF000DF91CF91089589E794E00E94C807809110
:101E0000EF01811109C00E9483120E94E0128091AB
:101E1000E20084608093E200089585E794E00E94E8
:101E2000C8071092EF01089581E794E00C94C80769
:101E30008DE694E00E94C8070C94972C89E694E004
:101E40000E94C8070E945D220E949D2C0E94851559
:101E50000C94B70D20915B012F5F822F62E30E94EB
:101E60000B2E992319F020935B01089510925B01CA
:101E700080915C01882371F18091F001843041F5FB
:101E80008091E9008F702091EC00922F917020FDDD
:101E900090E8892B94E09093E9009091EB0090FFFB
:101EA00014C09091EE0097FF10C09091E80095FF4C
:101EB00003C01092F100F9CF9091E80090FF05C0A7
:101EC0009091E8009E779093E8008F708093E900EE
:101ED00010925C01089542E061EC81E00E94FD11E6
:101EE00042E061EC82E00E94FD1142E061EC83E09F
:101EF0000E94FD1142E261EC84E00E94FD1142E18A
:101F000061EC85E00C94FD118091F201833009F4BD
:101F100055C030F4813071F0823009F48EC00895DC
:101F20008A3009F47AC08B3009F460C0893009F036
:101F30009CC020C08091F101813A09F096C0809147
:101F4000E800877F8093E8008091F5019091F60189
:101F5000892B21F460E18DE591E003C060E080E031
:101F600090E070E00E9439118091E8008B778093B7
:101F7000E80008958091F101813209F076C08091E6
:101F8000F5019091F601009719F0049709F06DC0E2
:101F90008091E800877F8093E8008091E80082FDCF
:101FA00005C08091F0018111F8CF5FC08091F100F0
:101FB00080936D018091E8008B7753C08091F1018F
:101FC000813A09F052C08091F5019091F601892B78
:101FD00009F04BC08091E800877F8093E8008091F2
:101FE000E80080FFFCCF80910C0136C08091F101A8
:101FF0008132D9F58091F5019091F601892BA9F5EF
:102000008091E800877F8093E8000E9432128091DF
:10201000F30180930C010C94611B8091F1018132DA
:1020200021F58091E800877F8093E8000E943212BA
:102030008091F40180936E0108958091F101813ABD
:10204000A1F48091E800877F8093E8008091E80008
:1020500080FFFCCF80916E018093F1008091E800B9
:102060008E778093E8000C943212089584B7877FAE
:1020700084BF88E10FB6F8948093600010926000EE
:102080000FBE90E080E80FB6F894809361009093C3
:1020900061000FBE0E9412160E9483120E94E0127D
:1020A0008091E20084608093E2008BEB9DE00E94CF
:1020B0009C2178940E9465150E94141682E091E09C
:1020C0000E9480150E94852C88E594E00E94C80734
:1020D0008091F001853089F484E594E00E94C8077E
:1020E0000E9421228091EE01882391F30E944922CF
:1020F000882371F30E94D810EBCF0E944216E8CFDC
:10210000292F332723303105C9F064F421303105FC
:1021100081F02230310509F043C08DE890E021EBD9
:1021200034E042C021323105F1F02232310541F173
:1021300037C082E190E02EE335E036C09927813048
:10214000910541F08230910541F0892B49F5EDEA86
:10215000F4E005C0E5E9F4E002C0EDE7F4E08491C5
:1021600090E09F0121C06530D8F4E62FF0E0EE0F3B
:10217000FF1FEB5DFE4F2081318189E090E014C0AC
:10218000653070F470E0FB01EE0FFF1FE55EFE4F5F
:1021900020813181FB01EA5EFE4F808190E004C026
:1021A00080E090E020E030E0FA0131832083089560
:1021B00080E189BD82E189BD09B400FEFDCF809137
:1021C000D8008F7D8093D8008091E000826080935A
:1021D000E0008091E00081FDFCCF0895CF92DF9276
:1021E000EF92FF920F931F93CF93DF93EC018B013C
:1021F0006A010E945112811133C0C114D10439F017
:10220000F60180819181081B190BC80FD91FE12CA1
:10221000F12C0115110519F18091E80085FD16C01A
:102220008091E8008E778093E800C114D10449F0D2
:10223000F60180819181E80EF91EF182E08285E04D
:102240000FC00E945112882321F30AC08991809304
:10225000F10001501109FFEFEF1AFF0ADACF80E019
:10226000DF91CF911F910F91FF90EF90DF90CF9072
:1022700008952091F7013091F8012617370748F0AB
:102280006115710539F42091E8002E772093E8005C
:1022900001C0B90140E061157105A9F12091F0017B
:1022A000222309F443C0253009F442C02091E800FC
:1022B00023FD40C02091E80022FD32C02091E800BB
:1022C00020FFE9CF4091F3002091F20030E0342B61
:1022D000FC01CF016115710559F02830310540F43A
:1022E00081918093F100615071092F5F3F4FF1CFD1
:1022F00041E02830310509F040E02091E8002E77D8
:102300002093E800C8CF4111C9CF0AC08091F001E5
:10231000882361F0853061F08091E80083FD0AC078
:102320008091E80082FFF2CF80E0089582E0089576
:1023300083E0089581E008952091F7013091F8013C
:102340002617370748F06115710539F42091E80028
:102350002E772093E80001C0B901FC0120E061154F
:10236000710591F18091F001882309F440C0853016
:1023700009F43FC08091E80083FD3DC08091E800F2
:1023800082FD2FC08091E80080FFE9CF2091F3000B
:102390008091F20090E0922B6115710559F0883020
:1023A000910540F424912093F10031966150710918
:1023B0000196F2CF21E0089709F020E08091E80033
:1023C0008E778093E800CBCF2111CCCF0AC08091CB
:1023D000F001882361F0853061F08091E80083FD91
:1023E0000AC08091E80082FFF2CF80E0089582E089
:1023F000089583E0089581E00895982F973058F567
:102400009093E900981739F07091EC002091ED005D
:102410005091F00003C0242F762F50E021FF19C007
:102420003091EB003E7F3093EB003091ED003D7F2B
:102430003093ED003091EB0031603093EB007093FE
:10244000EC002093ED005093F0002091EE0027FF68
:1024500007C09F5FD3CF8F708093E90081E008951C
:1024600080E008958091F10187FF11C08091E8001C
:1024700082FD05C08091F0018111F8CF11C08091DB
:10248000E8008B770BC08091F001882349F08091A0
:10249000E80080FFF8CF8091E8008E778093E80015
:1024A00008952091E4003091E50095E64091EC001C
:1024B000842F817040FF22C08091E80080FD1CC005
:1024C0008091F001882391F0853091F08091EB00AC
:1024D00085FD10C04091E4005091E500421753077C
:1024E00029F39A01915011F784E0089582E008954C
:1024F00083E0089581E0089580E008954091E80028
:1025000042FFDECF08950E94F1120E94F912E0EE20
:10251000F0E0808181608083E8EDF0E080818F775A
:10252000808319BCA7EDB0E08C918E7F8C93808165
:102530008F7E80831092EF0108950F931F93CF93A6
:10254000DF930E94F1120E94F912C8EDD0E0888159
:102550008F77888388818068888388818F7D88834E
:1025600019BC1092F0011092EC011092EE01109241
:10257000ED0100EE10E0F80180818B7F808388817F
:102580008160888342E060E080E00E94FD11E1EE1E
:10259000F0E080818E7F8083E2EEF0E080818160D8
:1025A0008083808188608083F80180818E7F808332
:1025B000888180618883DF91CF911F910F91089569
:1025C000E8EDF0E080818F7E8083E7EDF0E08081B0
:1025D0008160808384E082BF81E08093EF010C946E
:1025E0009D12E8EDF0E080818E7F80831092E20002
:1025F00008951092DA001092E10008951F920F9250
:102600000FB60F9211242F933F934F935F936F93C5
:102610007F938F939F93AF93BF93EF93FF9380919B
:10262000E10082FF0BC08091E20082FF07C0809131
:10263000E1008B7F8093E1000E942A0F8091DA00F5
:1026400080FF1FC08091D80080FF1BC08091DA00FE
:102650008E7F8093DA008091D90080FF0DC080E1E9
:1026600089BD82E189BD09B400FEFDCF81E0809380
:10267000F0010E94FB0E05C019BC1092F0010E94EF
:102680000D0F8091E10080FF19C08091E20080FF72
:1026900015C08091E2008E7F8093E2008091E2007D
:1026A00080618093E2008091D80080628093D8009E
:1026B00019BC85E08093F0010E94180F8091E10021
:1026C00084FF30C08091E20084FF2CC080E189BD8E
:1026D00082E189BD09B400FEFDCF8091D8008F7DD5
:1026E0008093D8008091E1008F7E8093E1008091FB
:1026F000E2008F7E8093E2008091E200816080930F
:10270000E2008091EC01882311F084E007C0809101
:10271000E30087FD02C081E001C083E08093F00107
:102720000E941E0F8091E10083FF29C08091E2008A
:1027300083FF25C08091E100877F8093E10082E0E4
:102740008093F0011092EC018091E1008E7F8093E4
:10275000E1008091E2008E7F8093E2008091E200B0
:1027600080618093E20042E060E080E00E94FD1121
:102770008091F00088608093F0000E94140FFF9118
:10278000EF91BF91AF919F918F917F916F915F91E9
:102790004F913F912F910F900FBE0F901F90189562
:1027A0001F920F920FB60F9211242F933F934F93C6
:1027B0005F936F937F938F939F93AF93BF93CF93C9
:1027C000DF93EF93FF93C091E900CF708091EC000D
:1027D000D82FD17080FDD0E81092E9008091F000F0
:1027E000877F8093F00078940E9414141092E9007F
:1027F0008091F00088608093F000CD2BCF70C09363
:10280000E900FF91EF91DF91CF91BF91AF919F913F
:102810008F917F916F915F914F913F912F910F9089
:102820000FBE0F901F9018951F93CF93DF93CDB7D6
:10283000DEB7AA970FB6F894DEBF0FBECDBFE1EFAB
:10284000F1E088E08E0F9091F10091938E13FBCF11
:102850000E94840F8091E80083FF1FC18091F101E5
:102860009091F201492F50E04A30510508F015C10E
:10287000FA01EA5AFF4F0C942B2E803881F08238EF
:1028800009F00BC18091F5018F708093E900809170
:10289000EB0085FB882780F91092E90006C0809143
:1028A000ED019091EE01911182609091E800977F87
:1028B0009093E8008093F1001092F100C8C0282F97
:1028C0002D7F09F0EAC0882319F0823061F0E5C05D
:1028D0008091F301813009F0E0C0933009F080E08D
:1028E0008093EE012BC08091F301811127C080916C
:1028F000F5018F7009F4D1C08093E9002091EB00BD
:1029000020FF1CC0933021F48091EB00806214C042
:102910009091EB0090619093EB0021E030E0A901F1
:1029200002C0440F551F8A95E2F74093EA001092C7
:10293000EA008091EB0088608093EB001092E90040
:102940008091E800877F86C08111A7C01091F301B4
:102950001F778091E3008078812B8093E300809142
:10296000E800877F8093E8000E9432128091E8009F
:1029700080FFFCCF8091E30080688093E300111119
:1029800002C082E001C083E08093F00186C08058DD
:10299000823008F082C08091F3019091F4018C3D67
:1029A00053E0950779F583E08A838AE289834FB7FC
:1029B000F894DE01139620E03EE051E2E32FF0E0D0
:1029C00050935700E49120FF03C0E295EF703F5F02
:1029D000EF708E2F90E0EA3010F0C79601C0C096DD
:1029E0008D939D932F5F243149F74FBF8091E8006D
:1029F000877F8093E8006AE270E0CE0101960E9432
:102A0000391114C0AE014F5F5F4F6091F5010E9414
:102A10008010BC01892B09F440C09091E800977F99
:102A20009093E80089819A810E949C118091E8002E
:102A30008B778093E80031C0803879F58091E80089
:102A4000877F8093E8008091EC018093F100809172
:102A5000E8008E778093E8000E9432121EC0811138
:102A60001CC09091F3019230C0F48091E800877F00
:102A70008093E8009093EC010E9432128091EC0167
:102A8000811106C08091E30087FD02C081E001C092
:102A900084E08093F0010E946B0F8091E80083FF37
:102AA0000AC08091E800877F8093E8008091EB0066
:102AB00080628093EB00AA960FB6F894DEBF0FBE3B
:102AC000CDBFDF91CF911F910895CF938091F001F9
:102AD0008823A1F0C091E900CF709091EC00892F7C
:102AE000817090FD80E8C82B1092E9008091E80089
:102AF00083FD0E941414CF70C093E900CF91089514
:102B000090937401809373010895E0917301F091A3
:102B10007401309721F00190F081E02D099480E05C
:102B20000895EF92FF920F931F93CF93DF93E0915D
:102B30007301F09174013097B1F18C010280F3813F
:102B4000E02D09958091D70182FF2DC080FF04C040
:102B500083E796E00E94C807E80110E18DE6E82EC1
:102B600086E0F82E8091D70180FF0BC088811F92EC
:102B70008F93FF92EF920E9461080F900F900F9039
:102B80000F90115021961111EDCF8091D70180FF48
:102B90000AC08BE696E0DF91CF911F910F91FF90D5
:102BA000EF900C94C807DF91CF911F910F91FF9088
:102BB000EF900895E0917301F0917401309721F046
:102BC0000480F581E02D09940895209171013091E0
:102BD00072018217930771F09093720180937101D3
:102BE000E0917301F0917401309721F00680F78134
:102BF000E02D0994089520916F01309170018217A2
:102C0000930771F09093700180936F01E0917301CD
:102C1000F0917401309721F00084F185E02D099442
:102C2000089508950C9411160E9463220E940C0AC4
:102C30000C942923CF93C82F8091D70182FF1EC007
:102C400080FF04C08CE896E00E94C8078091D701FD
:102C500080FF0CC01F92CF9387E896E09F938F93DD
:102C60000E9461080F900F900F900F908091D701F4
:102C700080FF04C085E896E00E94C8078C2FCF91A2
:102C80000C94B70DCF92DF92EF92FF920F931F93A8
:102C9000CF93DF93CDB7DEB72B970FB6F894DEBF97
:102CA0000FBECDBF0E94290A86E7C82E81E0D82E2C
:102CB00000E010E0E02E802F0E94550BF6014191BC
:102CC0006F01F42EF826B1F40F5F1F4F0E3011057F
:102CD00089F78FEF89838A831B820E946C2281602F
:102CE000782F9D838C8349815A816B818D810E94CD
:102CF000E51640C09091D70191FF04C08B870E94D8
:102D00005B0B8B8520E030E04F2D50E0922FBA0115
:102D1000022E02C0759567950A94E2F760FF24C001
:102D20002E83EF8221E030E0690102C0CC0CDD1C73
:102D30009A95E2F790E08C219D21892B09F420E0FF
:102D400028870E946C228160782F9A8789874E811C
:102D50005F8168858A850E94E516F801EA58FE4F72
:102D60008081C826C08206C02F5F3F4F26303105C4
:102D700069F6AACF0E949A26109175010E948515C6
:102D80001817A1F00E948515809375012B960FB638
:102D9000F894DEBF0FBECDBFDF91CF911F910F9191
:102DA000FF90EF90DF90CF900C941A162B960FB6F1
:102DB000F894DEBF0FBECDBFDF91CF911F910F9171
:102DC000FF90EF90DF90CF900895CF93DF93CDB732
:102DD000DEB72B970FB6F894DEBF0FBECDBF4F8383
:102DE000588769877A878B87DE01119686E0FD0117
:102DF00011928A95E9F785E0FE01379601900D92D0
:102E00008A95E1F749815A816B817C818D819E8110
:102E10000E94FB1D2B960FB6F894DEBF0FBECDBFF0
:102E2000DF91CF910895CF93882309F4C2C0C82FB2
:102E3000823859F40E94851581FDBBC089E30E9448
:102E400097200E94762189E30CC0833879F40E9490
:102E5000851580FDAEC083E50E9497200E947621F3
:102E600083E50E94EA20CF910C947621843859F4AE
:102E70000E94851582FD9DC087E40E9497200E94D4
:102E8000762187E4EECF8CEF8C0F813A48F48C2FBB
:102E90000E942D2B81118DC08C2F0E949720E3CF93
:102EA00080E28C0F883048F4C77081E001C0880F41
:102EB000CA95EAF70E943F21D6CF8BE58C0F83306D
:102EC00078F4C53A29F0C63A31F083E890E005C0BD
:102ED00081E890E002C082E890E0CF910C94E51583
:102EE00088E58C0F833108F064C0C83A39F1C93ADB
:102EF00041F1CA3A49F1CB3A51F1CC3A59F1CD3AC4
:102F000061F1C03B69F1CE3A71F1CF3A79F1C13B41
:102F100081F1C23B89F1C33B91F1C43B99F1C53BBF
:102F2000A1F1C63BA9F1C73BB1F1C83BB9F1C93B1F
:102F3000C1F1CA3BC9F180E090E038C082EE90E078
:102F400035C089EE90E032C08AEE90E02FC085EB6C
:102F500090E02CC086EB90E029C087EB90E026C083
:102F60008CEC90E023C08DEC90E020C083E891E0F1
:102F70001DC08AE891E01AC082E991E017C084E997
:102F800091E014C081E292E011C083E292E00EC0B1
:102F900084E292E00BC085E292E008C086E292E013
:102FA00005C087E292E002C08AE292E0CF910C94E1
:102FB000FB15CF910895882309F44BC0823859F44A
:102FC0000E94851581FF45C089E30E9497200E94D9
:102FD000762189E30CC0833871F40E94851580FF47
:102FE00038C083E50E9497200E94762183E50E94E5
:102FF000EA200C947621843859F40E94851582FFCA
:1030000028C087E40E9497200E94762187E4EFCFB2
:103010009CEF980F913A58F390E2980F983050F443
:10302000877091E001C0990F8A95EAF7892F0E9475
:103030004521DFCF9BE5980F933020F480E090E0AE
:103040000C94E515885A833120F480E090E00C94CC
:10305000FB150895882321F00E943F210C947621CE
:103060000895882321F00E9445210C94762108952B
:10307000BF92CF92DF92EF92FF920F931F93CF9365
:10308000DF9300D000D000D0CDB7DEB725E0FC0143
:10309000DE01119601900D922A95E1F7FC01408125
:1030A00031810281258122952F7063817481672B84
:1030B00009F4E5C23F3F19F44F3F09F4E0C27C0137
:1030C00049833A8389819A812E830E945620182F42
:1030D000B92E0E9455200E941C1FEB2DE295EF7027
:1030E000F0E0E05AFF4F2E810C942B2E8B2D807F29
:1030F0009B2D9F70F92E882319F0F29480EFF8220F
:10310000002349F0FF2009F467C28F2D0E944F2150
:103110000E94762161C2812F0E94DB17FF2009F4F3
:10312000AEC28F2D0E94552126960FB6F894DEBFB1
:103130000FBECDBFDF91CF911F910F91FF90EF9008
:10314000DF90CF90BF900C9476213B2D307F8B2D5C
:103150008F70303211F08295807F112319F0113079
:1031600021F12CC00023B9F0222309F4A0C12130A1
:1031700009F09DC126960FB6F894DEBF0FBECDBFF5
:10318000DF91CF911F910F91FF90EF90DF90CF9043
:10319000BF900C945F21222319F0213009F46FC2F3
:1031A0008E830E9462218E8196C1002321F02230FD
:1031B00008F065C27CC1211162C28DC1002321F0DB
:1031C000222309F474C108C2222309F484C119C25C
:1031D0002B2D26952695237030E02115310521F001
:1031E00021303105D1F04BC2002321F0812F9B2DDE
:1031F000937002C080E090E026960FB6F894DEBF90
:103200000FBECDBFDF91CF911F910F91FF90EF9037
:10321000DF90CF90BF900C94E515002321F0812F13
:103220009B2D937002C080E090E026960FB6F89434
:10323000DEBF0FBECDBFDF91CF911F910F91FF90E9
:10324000EF90DF90CF90BF900C94FB15812F00235F
:1032500019F00E94202502C00E94882526960FB6EC
:10326000F894DEBF0FBECDBFDF91CF911F910F91BC
:10327000FF90EF90DF90CF90BF900C940D268B2D98
:10328000837009F07BC00111FAC1812F8295869568
:103290008770880F880F912F9F70C92ED12CE12C39
:1032A000F12C082E04C0CC0CDD1CEE1CFF1C0A9473
:1032B000D2F714FF12C04FE050E060E070E004C0AD
:1032C000440F551F661F771F8A95D2F7CB01BA01AD
:1032D000609570958095909503C060E070E0CB019B
:1032E0002B2D269526952370422F50E04230510514
:1032F000D9F04330510569F16C297D298E299F2928
:103300004130510551F126960FB6F894DEBF0FBE3D
:10331000CDBFDF91CF911F910F91FF90EF90DF9084
:10332000CF90BF900C94431F6C297D298E299F2933
:1033300026960FB6F894DEBF0FBECDBFDF91CF91BA
:103340001F910F91FF90EF90DF90CF90BF900C9462
:103350005F1F0E94431FC701B60126960FB6F8945F
:10336000DEBF0FBECDBFDF91CF911F910F91FF90B8
:10337000EF90DF90CF90BF900C94271F002319F09F
:103380008B2D817001C08695882309F478C1812F27
:10339000829586958770880F880F912F9F70C92E10
:1033A000D12CE12CF12C082E04C0CC0CDD1CEE1C21
:1033B000FF1C0A94D2F714FF12C04FE050E060E007
:1033C00070E004C0440F551F661F771F8A95D2F71F
:1033D000CB01BA01609570958095909503C060E02F
:1033E00070E0CB012B2D269526952370422F50E0BF
:1033F00042305105D9F04330510569F16C297D29DE
:103400008E299F294130510551F126960FB6F89427
:10341000DEBF0FBECDBFDF91CF911F910F91FF9007
:10342000EF90DF90CF90BF900C941D206C297D29E8
:103430008E299F2926960FB6F894DEBF0FBECDBF0A
:10344000DF91CF911F910F91FF90EF90DF90CF9080
:10345000BF900C9439200E941D20C701B60126960A
:103460000FB6F894DEBF0FBECDBFDF91CF911F9195
:103470000F91FF90EF90DF90CF90BF900C940120C0
:10348000103FD1F118F4103E50F4A1C0123F09F4DE
:1034900063C008F44CC0133F09F473C098C01F7098
:1034A0008B2D8F710023A1F00E949A1F812F2696E9
:1034B0000FB6F894DEBF0FBECDBFDF91CF911F9145
:1034C0000F91FF90EF90DF90CF90BF900C942A184F
:1034D0000E94BB1F812F26960FB6F894DEBF0FBE49
:1034E000CDBFDF91CF911F910F91FF90EF90DF90B3
:1034F000CF90BF900C9431180023A9F02111BFC0C8
:103500008B2D8F7126960FB6F894DEBF0FBECDBF00
:10351000DF91CF911F910F91FF90EF90DF90CF90AF
:10352000BF900C94E01F223008F0A9C0E9CF00231F
:10353000A9F08B2D8F7126960FB6F894DEBF0FBEC3
:10354000CDBFDF91CF911F910F91FF90EF90DF9052
:10355000CF90BF900C949A1F002359F38B2D8F713D
:1035600026960FB6F894DEBF0FBECDBFDF91CF9188
:103570001F910F91FF90EF90DF90CF90BF900C9430
:10358000BB1F002399F08B2D8F7126960FB6F894F0
:10359000DEBF0FBECDBFDF91CF911F910F91FF9086
:1035A000EF90DF90CF90BF900C94851F26960FB6BA
:1035B000F894DEBF0FBECDBFDF91CF911F910F9169
:1035C000FF90EF90DF90CF90BF900C947B1F002373
:1035D000A9F0222309F4ADCF812F26960FB6F894D7
:1035E000DEBF0FBECDBFDF91CF911F910F91FF9036
:1035F000EF90DF90CF90BF900C941317222309F423
:10360000ADCF812F26960FB6F894DEBF0FBECDBF8B
:10361000DF91CF911F910F91FF90EF90DF90CF90AE
:10362000BF900C94DB174B2D4F70612FC7010E9488
:103630006A0826960FB6F894DEBF0FBECDBFDF91A5
:10364000CF911F910F91FF90EF90DF90CF90BF909F
:103650000C949F1E4B2D4F70612FC70126960FB6FD
:10366000F894DEBF0FBECDBFDF91CF911F910F91B8
:10367000FF90EF90DF90CF90BF900C94610C269656
:103680000FB6F894DEBF0FBECDBFDF91CF911F9173
:103690000F91FF90EF90DF90CF90BF9008950E9420
:1036A0005C210E9431210E9476210E9440270E94C5
:1036B0000D2680E090E00E94E51580E090E00C94FB
:1036C000FB150E944C210C944F1B0E945620292F61
:1036D00022952F7030E02C3031054CF42A30310522
:1036E0006CF4225031092230310588F407C02C30A7
:1036F000310549F02F30310531F009C0803E48F0E6
:10370000803F29F406C093FB882780F9089580E064
:10371000089581E00895CF93DF9300D000D01F92E9
:10372000CDB7DEB70F900F900F900F900F90DF91F5
:10373000CF910895CF93DF9300D000D000D0CDB7C4
:10374000DEB726960FB6F894DEBF0FBECDBFDF9171
:10375000CF9108951F93CF93DF93C091840116E01A
:1037600080918501C81799F0D0E01C9FF0011D9F42
:10377000F00D1124EA57FE4F40815181628173811F
:10378000848195810E949A1B2196C770E9CFDF91B1
:10379000CF911F9108954091B6015091B70160916A
:1037A000B8017091B9018091BA019091BB010C945C
:1037B0009A1B8091BB0182958F7009F054C0809153
:1037C000B801882309F44FC080918401A09185013C
:1037D0006091B6017091B7014091B9015091BA0161
:1037E000B6E08A1709F43FC090E041155105C1F1D8
:1037F0007F3F11F46F3FA1F1B89FF001B99FF00D29
:103800001124EA57FE4F218172132AC020816213CE
:1038100027C02281211124C0238134812417350738
:1038200010F421503109241B350B283C3105C0F41C
:103830002091BB012F7020612093BB0126E0289FBF
:10384000F001299FF00D1124E557FE4F80818F7004
:103850008061808386EB91E00E9438180C94AA1B4B
:1038600001968770BECF0895CF92DF92EF92FF92BC
:103870000F931F93CF93DF93CDB7DEB762970FB649
:10388000F894DEBF0FBECDBF8C0185E0F801DE01EC
:103890001D9601900D928A95E1F7D8014C911196F1
:1038A0005C91119712966C9112971396CD90DC90C3
:1038B00014973091B6017091B7018091B901909140
:1038C000BA01009709F46BC17F3F19F43F3F09F437
:1038D00066C1E090B801EE2009F4C0C02091BB01A0
:1038E000C816D90628F0F601E81BF90BCF0104C071
:1038F000809590958C0D9D1DFF24F394883C910537
:1039000078F0F12C207F09F0C6C07C2DD98AC88AB6
:1039100089890E948B1B86EB91E00E943818B1C008
:10392000822F807F09F046C0751314C0341312C073
:10393000611110C02F7020612093BB010E94CB1B2E
:1039400086EB91E00E9438188091BB01D801159652
:103950008C932EC0CD2819F15F3F11F44F3FF9F041
:10396000F62E61111CC0809184012091850136E002
:10397000821709F45AC090E0389FF001399FF00D8A
:103980001124EA57FE4F7181571306C07081471307
:1039900003C07281711103C001968770E9CFF62EC2
:1039A000662309F418C18091BB0181608093BB013B
:1039B000F12C11C1751308C0341306C0611104C085
:1039C0008091BB01D801C3C04D875E878D859E85E0
:1039D0006A8B0E94651B6A898823E1F16623D1F115
:1039E0002091BB01822F82958F7090E0029774F036
:1039F0008091B6019091B70198878F831986DB86F5
:103A0000CA862C87CE0107960E94381886E0F801F6
:103A1000A6EBB1E001900D928A95E1F70E94D91BC7
:103A20000E94CB1BFF24F394D6C04D875E878D8503
:103A30009E850E945620292F22952F7030E022303B
:103A400031050CF0BCC09F7009F0B6C0805E8830B4
:103A500008F4C1C0C8010E943818E4CFC816D906BE
:103A600008F453C0F601E81BF90BCF01883C91051F
:103A700008F450C0F12C7C2DD98AC88A89890E940B
:103A80008B1BE6EBF1E086E0DF011D928A95E9F7FA
:103A90000E94CB1BA0C0751314C0341312C0611157
:103AA00010C08091BB01F8018583C8010E943818BD
:103AB00086E0E6EBF1E0DF011D928A95E9F7FE2C46
:103AC0008AC04D875E878D859E856A8B0E94651BA7
:103AD0006A89882309F4BECF662309F4BBCF2091FD
:103AE000BB01822F82958F7090E002970CF48ECFED
:103AF0008091B6019091B7019A8389831B82DD8200
:103B0000CC822E83CE0101967FCF809590958C0D2F
:103B10009D1DACCFF62E662309F49CCF75132EC0E5
:103B200034132CC02091BB0120FD1FC0822F829531
:103B30008F70D9F0D80115962C9315978F3049F0D6
:103B40008F5F982F9295907F822F8F70892B15967B
:103B50008C93C8010E94381886E0F801A6EBB1E00A
:103B600001900D928A95E1F793CF86E0F801A6EBDC
:103B7000B1E001900D928A95E1F72DC04D875E87E7
:103B80008D859E850E94651B811140CF8091BB0170
:103B900081608093BB01C8010E9438181CC0662355
:103BA00009F458CF4D875E878D859E850E94651BE1
:103BB000882309F44FCF2ACF811148CF0CC024307D
:103BC00031050CF047CF9F7009F440CFF801958183
:103BD000907F09F03BCF8F2D62960FB6F894DEBF31
:103BE0000FBECDBFDF91CF911F910F91FF90EF904E
:103BF000DF90CF9008951F93CF93DF93CDB7DEB7BB
:103C00002C970FB6F894DEBF0FBECDBF4F835887F9
:103C100069877A878B879C87CE0107960E94341C20
:103C2000882369F08F8198852A853B85232BF1F1C4
:103C30009F3F09F063C08F3F09F060C037C086E046
:103C4000FE013796DE01119601900D928A95E1F7FB
:103C50006F817885EA85FB85309741F17F3F11F4CC
:103C60006F3F21F12091850130E0C90101968770F5
:103C700099274091840150E08417950709F447C0C3
:103C800069837A83FD83EC8396E0929FD001939FB2
:103C9000B00D1124AA57BE4FFE01319601900D922E
:103CA0009A95E1F7809385010E94AA1B16E0809106
:103CB0008401909185018917C1F1189FC0011124D9
:103CC0008A579E4F0E94341C882379F1E091840129
:103CD0001E9FF0011124EA57FE4F408151816281FD
:103CE0007381848195810E949A1B8091840190E068
:103CF00001968770992780938401D9CF4F81588589
:103D000069857A858B859C850E949A1BCFCF0E94FE
:103D1000611B1092850110928401E6EBF1E086E0D0
:103D2000DF011D928A95E9F7C1CF2C960FB6F89462
:103D3000DEBF0FBECDBFDF91CF911F910895EF92EF
:103D4000FF920F931F93CF93DF938C01892B09F47C
:103D50006CC0F12CEE24E394E8012196F8018491E3
:103D6000843740F4843008F051C0813081F08230D3
:103D700019F15BC0853709F444C0A8F19CE7980F9E
:103D8000903708F052C08F770E94DB1741C00E5F5A
:103D90001F4FFE01C49180E28C0F883048F4C77039
:103DA0008E2D01C0880FCA95EAF70E944F2114C0DA
:103DB0008C2F0E9413172DC00E5F1F4FFE01C49160
:103DC00080E28C0F883058F4C7708E2D01C0880FA8
:103DD000CA95EAF70E9455210E9476211AC08C2FBD
:103DE0000E94DB1716C00E5F1F4FFE01C491CC234B
:103DF00081F08FE99FE00197F1F700C00000C1500A
:103E0000F6CF0E5F1F4FFE01F49003C00E94131700
:103E10008E018F2D882309F49FCFEFE9FFE03197C2
:103E2000F1F700C000008150F5CFDF91CF911F91D5
:103E30000F91FF90EF90089508956093C0017093E3
:103E4000C1018093C2019093C3010C944F1B0F9347
:103E50001F930091C0011091C1012091C2013091C6
:103E6000C301DC01CB01802B912BA22BB32B8093C0
:103E7000C0019093C101A093C201B093C3011F91EF
:103E80000F910C944F1B0F931F930091C001109141
:103E9000C1012091C2013091C301DC01CB0180231B
:103EA0009123A223B3238093C0019093C101A093D7
:103EB000C201B093C3011F910F910C944F1B0F933C
:103EC0001F930091C0011091C1012091C201309156
:103ED000C301DC01CB0180279127A227B327809360
:103EE000C0019093C101A093C201B093C3011F917F
:103EF0000F910C944F1B1092BC011092BD011092B7
:103F0000BE011092BF010C944F1B41E050E060E0F5
:103F100070E004C0440F551F661F771F8A95D2F7C3
:103F20004093BC015093BD016093BE017093BF01EB
:103F30000C944F1B41E050E060E070E004C0440F7F
:103F4000551F661F771F8A95D2F78091BC0190910B
:103F5000BD01A091BE01B091BF01482B592B6A2B26
:103F60007B2B4093BC015093BD016093BE017093C5
:103F7000BF010C944F1B41E050E060E070E004C0D2
:103F8000440F551F661F771F8A95D2F740955095AD
:103F9000609570958091BC019091BD01A091BE018A
:103FA000B091BF01482359236A237B234093BC016E
:103FB0005093BD016093BE017093BF010C944F1BE1
:103FC00041E050E060E070E004C0440F551F661F00
:103FD000771F8A95D2F78091BC019091BD01A09185
:103FE000BE01B091BF01482759276A277B2740931C
:103FF000BC015093BD016093BE017093BF010C944E
:104000004F1B0F931F930091BC011091BD01209194
:10401000BE013091BF01DC01CB01802B912BA22B83
:10402000B32B8093BC019093BD01A093BE01B093CC
:10403000BF011F910F910C944F1B0F931F93009181
:10404000BC011091BD012091BE013091BF01DC0186
:10405000CB0180239123A223B3238093BC019093AF
:10406000BD01A093BE01B093BF011F910F910C94AD
:104070004F1B0F931F930091BC011091BD01209124
:10408000BE013091BF01DC01CB0180279127A2271F
:10409000B3278093BC019093BD01A093BE01B09360
:1040A000BF011F910F910C944F1B0895CF92DF9287
:1040B000EF92FF920F931F93CF93DF938C01C090E9
:1040C000C001D090C101E090C201F090C3014091C5
:1040D000BC015091BD016091BE017091BF01C42A25
:1040E000D52AE62AF72ACFE1D0E0D701C6010C2E67
:1040F00004C0B695A795979587950A94D2F780FF47
:1041000007C0B8018C2F0E94840C8130910531F4D6
:10411000219758F7B80180E00E94840CDF91CF917D
:104120001F910F91FF90EF90DF90CF9008959091A5
:104130000C01992321F090910D01911109C020915A
:104140000E0130910F01F90132969FEF40E030C02F
:10415000982F9695969596959F30A0F4E0910E0134
:10416000F0910F01E90FF11D877021E030E0A90106
:1041700002C0440F551F8A95E2F7CA019181892B2D
:10418000818308959091D70190FF23C01F928F9350
:104190008DEB96E09F938F930E9461080F900F9094
:1041A0000F900F9008959F3F39F04F5F4E3041F0D0
:1041B00051915813F8CF0DC05111F7CF942FF5CF6F
:1041C0009F3F39F0F901E90FF11D97FDFA958283C0
:1041D0000895089590910C01992321F090910D017B
:1041E000911109C020910E0130910F01F901329611
:1041F000205F3F4F30C0982F9695969596959F30AB
:10420000A8F4E0910E01F0910F01E90FF11D877004
:1042100021E030E0A90102C0440F551F8A95E2F762
:10422000CA01809591818923818308959091D70156
:1042300090FF16C01F928F938FE996E09F938F9304
:104240000E9461080F900F900F900F900895319683
:10425000E217F30729F090819813F9CF1082F7CF76
:10426000089581E090E0E0910E01F0910F01E80FD8
:10427000F91F1082019680319105A9F70895909158
:10428000D601892B8093D601089580959091D6010F
:1042900089238093D60108951092D60108959091B4
:1042A000D501892B8093D501089580959091D501F2
:1042B00089238093D50108951092D50108958093A4
:1042C000C40108951092C401089580910E01909147
:1042D0000F01FC0131969C01205F3F4F80E09191DE
:1042E00091118F5FE217F307D1F70895E0910E0166
:1042F000F0910F018091D6018083E0910E01F09141
:104300000F0190818091D501892B80838091C40118
:10431000882361F0E0910E01F0910F019081892BCB
:1043200080830E94652181111092C40180910E0149
:1043300090910F010C94911590933B0180933A0159
:104340000895CF92DF92EF92FF926C01EE24FF244A
:10435000C114D104E104F10421F0C701B60120E148
:1043600001C020E0C72ED82EE92EFF24C114D104AD
:10437000E104F10419F0285FC701B6016B017C016B
:1043800054E0F694E794D794C7945A95D1F7C114A2
:10439000D104E104F10419F02C5FC701B6016B01EF
:1043A0007C0142E0F694E794D794C7944A95D1F7FC
:1043B000C114D104E104F10419F02E5FC701B60164
:1043C000DC01CB01B695A79597958795892B8A2B0C
:1043D0008B2B09F02F5F822FFF90EF90DF90CF9013
:1043E00008958295982F9C7C392F36953695282FE5
:1043F000237344E0249FC0011124932F982B292F6D
:104400002A7A2695892F8575880F822B08951F9308
:10441000CF93DF931F92CDB7DEB799830E94F1212E
:10442000182F9981892F0E94F121212F30E0322FFE
:104430002227A901482BCA010F90DF91CF911F912C
:1044400008958091F001843009F11092D80120E4A0
:1044500088E190E00FB6F894A895809360000FBEB5
:104460002093600083B7817F846083BF83B78160BE
:1044700083BF7894889583B78E7F83BF88E10FB61A
:10448000F89480936000109260000FBE0895089524
:104490000895CF930E9447220E94290A0E94482231
:1044A000C0E08C2F0E94550B811104C0CF5FCE302D
:1044B000C1F701C081E0CF9108950E94611B0E9465
:1044C00085150C94B70D82E084BD93E095BD9AEFFD
:1044D00097BD80936E0008952FB7F8948091D9010D
:1044E0009091DA01A091DB01B091DC012FBF08951A
:1044F000CF92DF92EF92FF920F931F932FB7F89412
:104500004091D9015091DA016091DB017091DC0199
:104510002FBF6A017B01EE24FF248C0120E030E0F4
:10452000C016D106E206F30610F4415051099A0173
:10453000281B390BC9011F910F91FF90EF90DF905D
:10454000CF9008951F920F920FB60F9211248F9360
:104550009F93AF93BF938091D9019091DA01A0917D
:10456000DB01B091DC010196A11DB11D8093D90141
:104570009093DA01A093DB01B093DC01BF91AF917E
:104580009F918F910F900FBE0F901F9018950E94D2
:104590008312F8942FEF87EA91E6215080409040F3
:1045A000E1F700C0000087E090EBDC018093F901A7
:1045B0009093FA01A093FB01B093FC019CE088E189
:1045C0000FB6F894A895809360000FBE909360009A
:1045D000FFCFEF92FF920F931F93CF93DF93D82FCC
:1045E000C0E08C2F0E94550B00E010E0E82EF12C6B
:1045F000C701002E02C0959587950A94E2F780FDC9
:1046000006C00F5F1F4F0630110591F709C0602FDC
:104610007C2F80E00E94620CD813F3CF81E004C0AD
:10462000CF5FCE30F1F680E0DF91CF911F910F91F7
:10463000FF90EF900895CF93C82F8CE20E94E9225B
:10464000882321F08C2FCF910C94E92280E0CF9128
:104650000895CF930E947824811102C00E945E24A5
:1046600082EE96E00E94C807C5E6C15049F00E945C
:10467000290A8FE39CE90197F1F700C00000F5CF0C
:104680008BED96E00E94C80789E20E941B238111EE
:1046900013C18AE20E941B2381110E945E2485E0DF
:1046A0000E941B2381110E94C7220E9483248093B1
:1046B000D70187E00E941B238823A9F18BE10E9488
:1046C0001B23882351F08091D70181FB222720F9F9
:1046D00091E0922790FB81F90EC08EE00E941B238F
:1046E000882361F08091D70182FB222720F991E095
:1046F000922790FB82F98093D70115C080E10E9438
:104700001B239091D701882341F093FB222720F9A6
:1047100081E0822780FB93F904C0892F809580FB7C
:1047200090F99093D7018091D7010E9487240E942D
:1047300095248093EA0180EE0E941B23882341F098
:104740008091EA01982F909590FB80F98093EA017F
:1047500089E30E941B23882359F08091EA0181FBA1
:10476000222720F991E0922790FB81F98093EA01BA
:1047700082EE0E941B23882359F08091EA0182FB7C
:10478000222720F991E0922790FB82F98093EA0199
:1047900086EE0E941B23882359F08091EA0183FB57
:1047A000222720F991E0922790FB83F98093EA0178
:1047B00083EE0E941B23882359F08091EA0184FB39
:1047C000222720F991E0922790FB84F98093EA0157
:1047D00085E30E941B23882359F08091EA0185FB21
:1047E000222720F991E0922790FB85F98093EA0136
:1047F00081E30E941B23882359F08091EA0186FB04
:10480000222720F991E0922790FB86F98093EA0114
:1048100081E10E941B23882359F08091EA0187FBE4
:10482000222720F991E0922790FB87F98093EA01F3
:104830008091EA010E9499248091EA0187FB8827F0
:1048400080F980930D0187E20E941B23C82F8EE11F
:104850000E941B238111C2608FE10E941B238111E2
:10486000C46080E20E941B238111C86081E20E9423
:104870001B238111C06182E20E941B238111C0624F
:1048800083E20E941B238111C06484E20E941B23E7
:10489000882311F0C06802C0CC2329F08C2F0E941D
:1048A00090246C2F03C00E948C24682F70E080E05D
:1048B00090E0CF910C941D1FCF9108956DEE7EEF87
:1048C00080E090E00E94612E60E082E090E00E9433
:1048D000532E60E083E090E00E94532E60E084E07D
:1048E00090E00E94532E60E085E090E00C94532EFF
:1048F00080E090E00E944D2E21E08D3E9E4F09F019
:1049000020E0822F089582E090E00C94452E682FDD
:1049100082E090E00C94532E83E090E00C94452EBE
:10492000682F83E090E00C94532E84E090E00C9488
:10493000452E682F84E090E00C94532E8091DF0187
:1049400080FF0BC06091130185E0689FB0011124C6
:1049500075956795759567952BC081FF09C0609126
:10496000130185E0689FB00111247595679520C0FB
:1049700082FF07C06091130185E0689FB001112498
:1049800017C09091E0019923D1F060911201961720
:1049900088F72091130185E0289F90011124929FB0
:1049A000A001939F500D112470E0CA010E94172EA0
:1049B0006038710540F46115710539F002C065E099
:1049C00070E0862F08958FE7089581E00895809123
:1049D000DF0180FF08C06091110170E07595679557
:1049E0007595679521C081FF06C06091110170E047
:1049F0007595679519C082FF04C06091110170E040
:104A000010C09091E0019923C1F0609110019617B8
:104A1000A0F780911101899FC001112470E00E94CC
:104A2000172E6038710528F46115710521F0862F65
:104A300008958FE7089581E0089561E070E0F4CF74
:104A4000803F21F40E949E24819504C0813F29F477
:104A50000E949E248093E3010895823F21F40E94E6
:104A60009E24819504C0833F29F40E949E24809354
:104A7000E2010895893F19F40E94E72405C08A3FA6
:104A800031F40E94E72481958093E40108958B3FDF
:104A900021F40E94E724819504C08C3F29F40E94F0
:104AA000E7248093E5010895843F21F48091E1019A
:104AB000816017C0853F21F48091E101826011C0BF
:104AC000863F21F48091E10184600BC0873F21F48F
:104AD0008091E101886005C0883F31F48091E10157
:104AE00080618093E10108958D3F21F48091DF0181
:104AF00081600BC08E3F21F48091DF01826005C090
:104B00008F3F29F48091DF0184608093DF01089555
:104B1000803F39F48091E30187FF6CC01092E3017C
:104B200069C0813F29F48091E3011816BCF362C08B
:104B30009091E201823F29F497FF5CC01092E2015C
:104B400059C0833F19F41916CCF354C0893F41F47E
:104B50008091E40118160CF04DC01092E4014AC097
:104B60008A3F29F48091E40187FF44C0F6CF8B3F50
:104B700039F48091E50187FF3DC01092E5013AC00C
:104B80008C3F29F48091E5011816BCF333C0843FB3
:104B900021F48091E1018E7F17C0853F21F480913F
:104BA000E1018D7F11C0863F21F48091E1018B7F6F
:104BB0000BC0873F21F48091E101877F05C0883FCA
:104BC00031F48091E1018F7E8093E10113C08D3F2C
:104BD00021F48091DF018E7F0BC08E3F21F4809104
:104BE000DF018D7F05C08F3F29F48091DF018B7F2E
:104BF0008093DF018091E20181110EC08091E30179
:104C000081110AC08091E401811106C08091E50103
:104C1000811102C01092E00108958091D70183FFB5
:104C20007EC08EE197E00E94C8078091E1011F924B
:104C30008F9389E197E09F938F930E94610887E1AA
:104C400097E00E94C8078091E201282F332727FDB3
:104C500030953F938F9384E197E09F938F930E94C9
:104C6000610882E197E00E94C8078091E301282F44
:104C7000332727FD30953F938F938FE097E09F93E5
:104C80008F930E9461088DE097E00E94C807809191
:104C9000E401282F332727FD30953F938F938AE037
:104CA00097E09F938F930E94610888E097E00E94AD
:104CB000C8078091E501282F332727FD30953F93C2
:104CC0008F9385E097E09F938F930E94610882E025
:104CD00097E00E94C8078091E0011F928F938FEFA9
:104CE00096E09F938F930E9461088DEF96E00E945B
:104CF000C8078091DF011F928F938AEF96E09F9300
:104D00008F930E94610887EF96E00E94C8078DB7D5
:104D10009EB74C960FB6F8949EBF0FBE8DBF81EE26
:104D200091E00E94DA150E946C229093DE0180933C
:104D3000DD0108951F93CF93DF938091DD01909162
:104D4000DE010E947822AC019091E001992321F0CC
:104D50002091140130E006C0209115018AE0289FBF
:104D6000900111244217530708F486C08091E20194
:104D7000C091E301D091E4011091E501811107C0D8
:104D8000C11176C0D11174C0111172C075C09F3F9E
:104D900019F09F5F9093E001181624F40E949E245E
:104DA0008093E2018091E20187FF05C00E949E246A
:104DB00081958093E2011C1624F40E949E24809326
:104DC000E3018091E30187FF05C00E949E24819545
:104DD0008093E3016091E201662339F1C091E30120
:104DE000CC2319F1772767FD7095872F972F0E94A5
:104DF0001C2D23E333E343E35FE30E94802D0E94F5
:104E0000E92C6093E2016C2F772767FD7095872F5F
:104E1000972F0E941C2D23E333E343E35FE30E94BB
:104E2000802D0E94E92C6093E3011D1624F40E945A
:104E3000E7248093E4018091E40187FF05C00E948C
:104E4000E72481958093E401111624F40E94E7245D
:104E50008093E5018091E50187FF05C00E94E7246A
:104E600081958093E501DF91CF911F910C940D26E0
:104E70009F3F09F08ECF96CFDF91CF911F9108957C
:104E8000E1EEF1E085E0DF011D928A95E9F71092ED
:104E9000E0011092DF01089581E499E00E94C807C3
:104EA0001F9281E08F931F9285E08F9383EF98E0AC
:104EB0009F938F930E9461080F900F900F900F9017
:104EC0000F900F9008958330E9F128F4813061F05C
:104ED000823009F10895853009F462C008F449C0B0
:104EE000863009F474C0089580911501262F30E0B2
:104EF000280F311D2F3F310524F4680F60931501F1
:104F000003C08FEF80931501809115011F928F933D
:104F10008CE298E072C080911401262F30E0280FB7
:104F2000311D2F3F310524F4680F6093140103C035
:104F30008FEF80931401809114011F928F938AE167
:104F400098E05BC080911301262F30E0280F311DBF
:104F50002F3F310524F4680F6093130103C08FEFD6
:104F600080931301809113011F928F9387E098E043
:104F700044C080911201262F30E0280F311D2F3FB1
:104F8000310524F4680F6093120103C08FEF809302
:104F90001201809112011F928F9382EF97E02DC032
:104FA00080911101262F30E0280F311D2F3F310550
:104FB00024F4680F6093110103C08FEF80931101F7
:104FC000809111011F928F9389ED97E016C0809117
:104FD0001001262F30E0280F311D2F3F310524F41A
:104FE000680F6093100103C08FEF809310018091D0
:104FF00010011F928F938EEB97E09F938F930E94E7
:1050000061080F900F900F900F900895833081F1F9
:1050100028F4813059F08230D1F00895853009F4B8
:1050200049C0B8F1863009F456C008958091150141
:10503000681720F4861B8093150102C01092150199
:10504000809115011F928F938FEA97E054C0809151
:105050001401681720F4861B8093140102C010927B
:105060001401809114011F928F938DE997E043C042
:1050700080911301681720F4861B8093130102C0EE
:1050800010921301809113011F928F938AE897E089
:1050900032C080911201681720F4861B80931201A0
:1050A00002C010921201809112011F928F9385E726
:1050B00097E021C080911101681720F4861B80932E
:1050C000110102C010921101809111011F928F9362
:1050D0008CE597E010C080911001681720F4861BC2
:1050E0008093100102C010921001809110011F9254
:1050F0008F9381E497E09F938F930E9461080F90B4
:105100000F900F900F900895CF93C82F1F928F93F9
:1051100086E49AE09F938F930E94610881E090E07B
:10512000A0E0B0E0BC01CD0104C0660F771F881F6E
:10513000991FCA95D2F70E941D1F0F900F900F90D4
:105140000F90CF910C94611BCF938D3109F465C002
:10515000B0F58E3009F4CCC100F5873009F49BC15D
:10516000A8F4863009F06DC28091D701817F8E7FCF
:105170008093D7018BE49AE00E94C8078DE89EE0F7
:105180000E94C80781E08093E70180C1883009F45C
:105190004FC08B3009F47CC154C2863109F4F0C190
:1051A00038F4803109F4B8C1813109F430C249C200
:1051B000893109F4CEC18B3109F486C142C28533ED
:1051C00009F437C248F4873209F433C208F433C211
:1051D000893209F42EC235C2833438F48A3308F098
:1051E0002CC2883309F454C12CC2833409F421C27F
:1051F000883409F026C20E94611B8CE79EE00E9461
:10520000C8079FEF23ED80E3915020408040E1F7F5
:1052100000C000000E94C72239C18CE99EE00E94B4
:10522000C8070E94A32C0E9485150E94B70D2EC1AD
:1052300081E99EE00E94C8078CE59CE00E94C807B7
:105240000E948C241F928F9389E59CE09F938F93FB
:105250000E94610887E59CE00E94C8070E948324A1
:10526000C82F84E49CE00E94C8071F92CF938FE36D
:105270009CE09F938F930E9461088DE39CE00E94C5
:10528000C80783E39CE00E94C8078C2F81701F929F
:105290008F9380E39CE09F938F930E9461088EE23E
:1052A0009CE00E94C80784E29CE00E94C807C1FB02
:1052B000882780F91F928F9381E29CE09F938F93C0
:1052C0000E9461088FE19CE00E94C80783E19CE096
:1052D0000E94C807C2FB882780F91F928F9380E144
:1052E0009CE09F938F930E9461088EE09CE00E9457
:1052F000C80785E09CE00E94C807C3FBCC27C0F923
:105300001F92CF9382E09CE09F938F930E9461084D
:1053100080E09CE00E94C8070E949524C82F8CEE74
:105320009BE00E94C8071F92CF9387EE9BE09F935C
:105330008F930E94610885EE9BE00E94C8078CEC69
:105340009BE00E94C8078C2F81701F928F9389EC7D
:105350009BE09F938F930E9461088DB79EB78096C4
:105360000FB6F8949EBF0FBE8DBF87EC9BE00E94E6
:10537000C80780EB9BE00E94C807C1FB882780F923
:105380001F928F938DEA9BE09F938F930E946108F9
:105390008BEA9BE00E94C80789E99BE00E94C8074E
:1053A000C2FB882780F91F928F9386E99BE09F9329
:1053B0008F930E94610884E99BE00E94C80782E8FD
:1053C0009BE00E94C807C3FB882780F91F928F9338
:1053D0008FE79BE09F938F930E9461088DE79BE08E
:1053E0000E94C80783E79BE00E94C807C4FB882788
:1053F00080F91F928F9380E79BE09F938F930E9489
:1054000061088EE69BE00E94C8078CE59BE00E9445
:10541000C807C5FB882780F91F928F9389E59BE019
:105420009F938F930E94610887E59BE00E94C807C5
:105430008BE39BE00E94C807C6FB882780F91F9278
:105440008F9388E39BE09F938F930E94610886E38C
:105450009BE00E94C8078EE29BE00E94C807C7FB42
:10546000CC27C0F91F92CF938BE29BE09F938F9341
:105470000E94610889E29BE00E94C8078DB79EB731
:105480004C960FB6F8949EBF0FBE8DBFC1E0DEC034
:1054900082E79AE05BC08091D701C82FC17080FF7E
:1054A00009C08FE69EE00E94C8078091D701817FE6
:1054B0008E7F47C083E69EE00E94C8078091D70197
:1054C00081608093D701E2CF9091D70191FBCC27E7
:1054D000C0F981E0C827892FC0FB81F98093D701EB
:1054E000CC2319F086E59EE027C088E49EE02EC01C
:1054F0009091D70192FBCC27C0F981E0C827892F72
:10550000C0FB82F98093D701CC2319F089E39EE098
:1055100013C089E29EE01AC09091D70193FBCC277B
:10552000C0F981E0C827892FC0FB83F98093D70198
:10553000CC2351F08DE19EE00E94C8078091D701F5
:1055400081608093D70182C080E19EE00E94C807FD
:105550009DCF81E09EE00E94C80785ED9DE00E94FE
:10556000C80788E99DE00E94C8078BE69DE00E947D
:10557000C80787E29DE00E94C8078CEF9CE0E6CF59
:105580008EEE9CE00E94C8070E9485151F928F93A3
:1055900084ED9CE09F938F930E94610880910C01A1
:1055A0001F928F938DEB9CE09F938F930E946108D5
:1055B00080916E011F928F938AEA9CE09F938F9354
:1055C0000E94610880910D011F928F9387E99CE0F2
:1055D0009F938F930E9461088091D9019091DA0185
:1055E000A091DB01B091DC01BF93AF939F938F93A8
:1055F00083E89CE09F938F930E9461088DB79EB7CC
:1056000046960FB6F8949EBF0FBE8DBF3FCF0E9447
:10561000611BC0910D0181E0C827C0930D01CC230F
:1056200029F089E79CE00E94C80710C08EE69CE044
:105630008DCF80E003C08D5101C089530E94842822
:1056400025CF8CE69CE00E94C807C0E08C2FCF914C
:10565000089580E0089580E00895CF93C82F809149
:10566000E701813081F020F0823009F44FC045C15C
:10567000E0910E01F0910F018081813169F0823259
:1056800009F03DC109C0E0910E01F0910F01808148
:10569000813111F0823261F48C2F0E94292B81110B
:1056A00004C08C2F0E94A4282FC081E090E02CC061
:1056B0008C2F0E942B2B811126C0C431E1F070F495
:1056C000CB3081F0C031D1F40E944C278EE39AE0B8
:1056D0000E94C80782E08093E70115C0C93259F0E3
:1056E000C83361F48BE49AE00E94C80782E49AE030
:1056F0000E94C80708C01092E70103C18CE39AE03A
:105700000E94C807FEC081E08170FDC0C43220F550
:10571000CE3108F0C0C0CB3099F1C8F4C73009F0E1
:10572000D2C08AE08093150194E19093140193E034
:10573000909313018093120188E08093110188E215
:105740008093100182EE98E00E94C807BFC0C33169
:1057500049F1C431C1F0B7C0CB3409F4A9C028F471
:10576000C93289F0C83361F0AEC0C13509F49EC0BA
:10577000C23509F499C0CE3409F0A5C06AE09EC0D4
:105780000E944C27A3C08091E601882319F0109253
:10579000E6019CC08FEE98E00E94C80781E08093EC
:1057A000E701B1C089EC98E00E94C80787EB98E058
:1057B0000E94C807809115011F928F9384EB98E097
:1057C0009F938F930E94610882EB98E00E94C80724
:1057D00080EA98E00E94C807809114011F928F937D
:1057E0008DE998E09F938F930E9461088BE998E080
:1057F0000E94C8078CE898E00E94C80780911301B6
:105800001F928F9389E898E09F938F930E9461087D
:1058100087E898E00E94C80786E798E00E94C807DA
:10582000809112011F928F9383E798E09F938F934B
:105830000E94610881E798E00E94C8078CE598E023
:105840000E94C807809111011F928F9389E598E00B
:105850009F938F930E94610887E598E00E94C80794
:1058600080E498E00E94C807809110011F928F93F6
:105870008DE398E09F938F930E9461088BE398E0FB
:105880000E94C8078DB79EB748960FB6F8949EBF82
:105890000FBE8DBF1BC0CE51EC2FF0E0E15DFE4F7F
:1058A00080818093E60112C061E003C061E006C020
:1058B0006AE08091E6010E94632708C08091E601BA
:1058C0000E94062803C080EE98E013C08091E60194
:1058D000882369F01F928F938AED98E09F938F93AE
:1058E0000E9461080F900F900F900F9004C087EDF9
:1058F00098E00E94C80781E006C01092E70180E0AE
:1059000002C080E001CFCF910895E1E8F0E080810E
:10591000886080838081816080838FB7F89493E072
:105920009093890090ED909388008FBF0895EFE6E3
:10593000F0E08081826080830895EFE6F0E080816E
:105940008D7F80830895EFE6F0E0908182E08927E3
:10595000808308951F920F920FB60F9211242F93F8
:105960003F934F935F936F937F938F939F93AF93E7
:10597000BF93EF93FF938091E8019091E901019625
:105980009093E9018093E801811103C082E00E94B5
:10599000B70DE091E901E695E695F0E0E455F14FA9
:1059A000E4918091E8018E1303C080E00E94B70D5E
:1059B000FF91EF91BF91AF919F918F917F916F91E7
:1059C0005F914F913F912F910F900FBE0F901F90BD
:1059D000189504D06894B1118DC0089570D088F0E6
:1059E0009F5790F0B92F9927B751A0F0D1F0660FCB
:1059F000771F881F991F1AF0BA95C9F712C0B130E6
:105A000081F077D0B1E0089574C0672F782F882790
:105A1000B85F39F0B93FCCF3869577956795B39524
:105A2000D9F73EF490958095709561957F4F8F4F93
:105A30009F4F0895E89409C097FB3EF49095809598
:105A4000709561957F4F8F4F9F4F9923A9F0F92F44
:105A500096E9BB279395F695879577956795B795C2
:105A6000F111F8CFFAF4BB0F11F460FF1BC06F5FA8
:105A70007F4F8F4F9F4F16C0882311F096E911C0BA
:105A8000772321F09EE8872F762F05C0662371F0DB
:105A900096E8862F70E060E02AF09A95660F771FEF
:105AA000881FDAF7880F9695879597F9089557FD1F
:105AB0009058440F551F59F05F3F71F04795880F7C
:105AC00097FB991F61F09F3F79F087950895121613
:105AD00013061406551FF2CF4695F1DF08C01616BF
:105AE00017061806991FF1CF869571056105089470
:105AF0000895E894BB2766277727CB0197F9089587
:105B00000BD078C069D028F06ED018F0952309F03A
:105B10005AC05FC01124EECFCADFA0F3959FD1F326
:105B2000950F50E0551F629FF001729FBB27F00D4B
:105B3000B11D639FAA27F00DB11DAA1F649F6627A0
:105B4000B00DA11D661F829F2227B00DA11D621FEF
:105B5000739FB00DA11D621F839FA00D611D221FA9
:105B6000749F3327A00D611D231F849F600D211D8D
:105B7000822F762F6A2F11249F5750408AF0E1F030
:105B800088234AF0EE0FFF1FBB1F661F771F881F79
:105B900091505040A9F79E3F510570F014C0AACF14
:105BA0005F3FECF3983EDCF3869577956795B79564
:105BB000F795E7959F5FC1F7FE2B880F911D96958E
:105BC000879597F9089597F99F6780E870E060E0FE
:105BD00008959FEF80EC089500240A941616170686
:105BE00018060906089500240A94121613061406CE
:105BF00005060895092E0394000C11F4882352F031
:105C0000BB0F40F4BF2B11F460FF04C06F5F7F4FE8
:105C10008F4F9F4F0895991B79E004C0991F9617E5
:105C200008F0961B881F7A95C9F78095089597FB11
:105C3000072E16F4009407D077FD09D00E94312E6C
:105C400007FC05D03EF4909581959F4F089570957F
:105C500061957F4F0895EE0FFF1F0590F491E02DA1
:105C60000994AA1BBB1B51E107C0AA1FBB1FA617A3
:105C7000B70710F0A61BB70B881F991F5A95A9F7F5
:105C800080959095BC01CD010895F999FECF92BD04
:105C900081BDF89A992780B50895A8E1B0E042E067
:105CA00050E00C94682E262FF999FECF1FBA92BDB2
:105CB00081BD20BD0FB6F894FA9AF99A0FBE0196ED
:105CC00008950E94532E272F0C94542EDC01CB01F3
:105CD000FC01F999FECF06C0F2BDE1BDF89A3196FC
:105CE00000B40D9241505040B8F70895F894FFCF9A
:105CF0002002B80DA90E860E520E1E0E0101C5011E
:105D000028080A03140A3F4D3620392C06DF05A95E
:105D10000589055005C304DC04F5040E052E0501B4
:0A5D2000020304050607080900004D
:00000001FF
